:060000001EC0FECF74C01B
:1000060090C145C1FACF79C07DC0F7CFF6CFF5CF05
:10001600F4CFF3CFF2CFF1CFF0CFEFCFEECFEDCFDE
:10002600F350CBD978B9BBF0FBF92B0B00080000D5
:100036000200020034000000F894EE27ECBBF1E069
:10004600FBBFEBBFE5BFF8E1F1BDE1BD8DE0A2E08E
:10005600BB27ED938A95E9F780E094E0A0E6ED935F
:100066000197E9F7E6E3F0E085919591009761F055
:10007600A591B59105901590BF01F00105900D92DF
:100086000197E1F7FB01F0CFEFE5EDBFE4E0EEBF4E
:10009600C0E6D1E057C1E5B7E063E5BFE5B7E06884
:1000A600E5BF889500000895EFE3E7BBE4BBE0E217
:1000B600E1BBE8E3E2BBE0E4E8B988EC90E0019755
:1000C600F1F7E0E0E2BF44245524EBE0EEBD0895ED
:1000D600E0E8E8B9E0E0EEBDE8BBE7BBE5BBE4BBC2
:1000E600E1BBE8E0E2BB0895EA93EFB7EA93E89450
:1000F60020F8EBB7EF774ED221C1EA93E0E0E5BBFB
:10010600E99118950A921A92FA926A937A938A93C7
:100116009A93AA93BA93EA93FA93EFB7EA933FD2E4
:10012600DF0140D2EF738E2FFD0144D2A1E0B0E093
:100136009CD2A091640144D2EA23FB23BF012FD2B3
:1001460039D2DB019BD2EE0FEE0FE82BE8BB27D2AC
:1001560029D2E07C37D29FD29AD2E5BB15B2E82DE0
:10016600EE5FA1E07AD2E129E5BBE3E08E1610F45A
:10017600839401C08824E3E0EB1521F425D2EAE05C
:100186002AD239C0E4E0EB1521F41ED2EBE023D2EB
:1001960032C0E5E0EB15E9F427D211F4ECE001C03A
:1001A600EDE0E0936001A09165010AD2E4E6F0E09B
:1001B6008AD2E09361011CD21ED2DF0121D2E093E4
:1001C600620116D2BB271CD2E0936301E0E01CD289
:1001D60012C0A72D10D2E0936001A72DBB2710D225
:1001E600E0936101A62D07D2E0936201A62DBB27FD
:1001F60007D2E0936301BB2021F5E0E005D290FC35
:1002060002C0E4E001D2E4E6F1E00F01A081E8B12A
:10021600E072D8D1F595E7953AD2EA2BD001EC9366
:10022600E6EAFFE04E165F0620F4F20131962F0152
:1002360008C0EBB7E068AED1689420F849DF68944F
:1002460026F8E1E0EB1511F4ECE0DED1E2E0EB1587
:1002560011F4E3E0D9D1EAE0AE1610F4A39409C094
:10026600AA24E894849B689421F8E894839B689474
:1002760022F8E991EFBFF991E991B991A991999184
:10028600899179916991F9901990099018951A9226
:10029600AA93BA93EA93FA93EFB7EA9320FE05C0BE
:1002A600E0E0E3BDE2B5E1FDFDCFEBE39E1610F421
:1002B60093942BC09924EBE36E1610F4639425C037
:1002C600662430FC03C094D1A03009F418C08CD148
:1002D60031F49DD1E4BDE2B5E2FDFDCF10C097D16A
:1002E60071D1AFEFB0E010D2EA1BFB0BE3BDE2B574
:1002F600E1FDFDCFE8B7E068E8BFE8EDE9BFE7E17B
:100306007E1610F4739401C0772420FE02C0689410
:1003160026F8E991EFBFF991E991B991A991199060
:100326001895EA93EFB7EA93E8E5E9BFE8B7E0681E
:10033600E8BFEFEFE4BDE2B5E2FDFDCFE991EFBF27
:10034600E9911895E0E0E8BBEFE3E7BBE0E0E5BB49
:10035600EFE3E4BBE8E3E2BBE0E2E1BBE0E0E3BFFE
:10036600E2BFEFBDEBE0EEBDE0E0EDBDECBDE7BD0D
:10037600E6BDEBBDECE9EABDE0E0E9BDE0E1E8BDE4
:10038600E8E0E2BDE5E0E5BDE0E0E4BDE3BDE8E5CB
:10039600E9BFE0E0EAB9E0E4E8B9E0E0E0BFE6B9E9
:1003A600EDB9E6BFE8EEF3E035D1A0E0B0E0B3D1B9
:1003B60034D1A1E0B0E0AFD133D11AD1A13F30F0B2
:1003C600E0E02BD1A0E0B0E0E0E0B1D1A091660181
:1003D600A23030F0E0E024D1A1E0B0E0E0E0A7D127
:1003E600789423FE05C0A0E020FCA1E0A03009F02F
:1003F60001C05ADE20FA23F820FCC5C024FC04C044
:1004060025FC02C021FC01C035C0CC24DD2421FE20
:1004160002C009D108F00DC0EAE0F0E0FBD0F60119
:1004260031966F014424552403D110F0E3E0BE2E2B
:10043600EECFFED010F0F7D008F00FC0689424F885
:10044600E0E0E5BDE2B5E0FDFDCFE0E0E4BDE2B50C
:10045600E2FDFDCF9924E1E0BE2EE5D028F0E4E0F0
:10046600BE2E689427F830F821FCFECFDCD010F0C1
:10047600E5E0BE2E24FE02C022FC01C009C0E7E171
:100486007E1610F4739401C07724ECE2F1E0C2D03A
:1004960024FE02C021FC01C008C0E89424F8689438
:1004A60025F8E2E0BE2E21FCFECF25FE02C022FC8E
:1004B60001C009C0EBE36E1610F4639401C0662414
:1004C600ECE2F1E0A7D025FE02C021FC01C012C07B
:1004D6009924E89425F8E0E0E4BDE2B5E2FDFDCF1D
:1004E600E5E0E5BDE2B5E0FDFDCF44245524BB249F
:1004F60021FCFECF27FE02C022FC01C02EC0CC2468
:10050600DD2422FE2AC070D061F472D0A03F20F410
:100516007ED0EF5F82D004C0E0EF7FD0E1E080D0F4
:100526000BC066D0A23020F072D0E15076D004C065
:10053600E0E073D0E0E074D0EBE0F0E0CE16DF064A
:1005460030F4F60131966F01ECE2F1E002C0E4E628
:10055600F0E0FA93EA9371D0D4CF27FE02C021FCD3
:1005660001C010C0E89427F852D0A0E0B0E0DFD078
:10057600E0916601A1E0B0E0DAD0E89430F8BB245F
:1005860021FCFECF05C026FE03C0E89426F883DDD5
:1005960028CFFFCFEBBFEAB7E068EABF0895E82DA2
:1005A600F0E00895E05AFE4FE081F0E0EA5DFF4F8B
:1005B600E4910895A3E0B0E0A7D0EA1BFB0B0895F1
:1005C600B0E00895F0E00895ECE0E0936001E5E026
:1005D600E09361010895E0936201ECE0E09363012A
:1005E600E0E0E09364010895E0916601E03008954B
:1005F600A09165010895E4DFEAE0F0E064D0089593
:10060600EAE0F0E065D00895E09364010895E09192
:1006160065010895FA93EA9310C0E0936501089581
:10062600E09366010895E4EFF1E0CE16DF06089543
:10063600E8ECF0E0CE16DF060895E991F9913096E0
:1006460039F080ED97E00197F1F7A8953197C9F752
:100656000895F195E195F0400895EE230E2EEA2FC8
:1006660019F0EE0F0A94E9F70895EE230E2EFD0118
:1006760021F0EE0FFF1F0A94E1F70895EE230E2EE8
:10068600FD0121F0F695E7950A94E1F70895F595B1
:10069600E795F595E795F595E795F595E795089529
:1006A6000024112490E1AA0FBB1F001C111C0E1A76
:1006B6001F0A18F40E0E1F1E01C0A1609A9599F725
:1006C600FD01D001089512D0EBDF0EF4C2DF0895CC
:1006D600E894B7FF04C0A095B09511966894F7FD0D
:1006E600B8DFDEDFFD010EF4B4DF0895E894F7FF0E
:1006F60002C0AFDF6894B7FF06C0A095B09511960B
:1007060000F8039400FA08951B2EBF2FF12D1A2E20
:10071600AE2FE12D0895E199FECFFF93FFB7F89430
:10072600AEBBBFBBE09AEDB3FFBFFF910895E19B5F
:1007360002C0A895FCCF9FB7F894AEBBBFBBE09AAA
:100746008DB3E81719F0EDBBE29AE19A9FBF0895C1
:00000001FF
